:100000000C94AF010C94E7010C94E7010C94E70108
:100010000C94E7010C94E7010C94E7010C94E701C0
:100020000C94E7010C94E7010C94BD1D0C948F1EF9
:100030000C94B1180C94E7010C94E7010C94E701BF
:100040000C94E7010C94E7010C94E7010C94E70190
:100050000C94E7010C9439190C94E7010C94E70116
:100060000C94E7010C94E7010C94E7010C94E70170
:100070000C94E7010C94E7010C94E7010C94E70160
:100080000C94E7010C94E7010C94E7010C94E70150
:100090000C94E7010C94E7010C94E7010C94E70140
:1000A0000C94E7010C94E7010C94E701AF04AF0452
:1000B000DB04DB0443056105790679066C0505065A
:1000C00016061606FC1E231F1B20231F1B206F1F56
:1000D000921F1B20E91FF81FA8001E001F00200010
:1000E00021002200230024002500260027002D00E7
:1000F0002E002A002A00290014001A00080015000A
:1001000017001C0018000C00120013002F00300014
:1001100031004C002B0039000400160007000900D4
:100120000A000B000D000E000F0033003400280001
:100130004B00E10031001D001B0006001900050006
:1001400011001000360037003800E50052004E0064
:100150000000E000E300E2002C002C002C00000076
:10016000E6000151E300500051004F004D00010036
:100170000100010001000100010001000100010077
:100180000100010001000100010001000100010067
:100190000100010001000100010001000100010057
:1001A0000100010001000100005C010001000100EC
:1001B0000100010001000100010001000100010037
:1001C0000100010001000100010001000100010027
:1001D0000100010001000100010001000100010017
:1001E0000100010001000000010001000100010008
:1001F00001000100000001000100010001000100F8
:1002000001000100380344006900730061007200BE
:100210007200610079002000280053007400610022
:1002200067006700650072006500640020004C00F4
:10023000610079006F00750074002900000012034E
:1002400053006E00650061006B0062006F00780073
:1002500000000403090409023B00020100A0FA099E
:1002600004000001030101000921110100012240E5
:1002700000070581030800010904010001030000D3
:1002800000092111010001227B00070582032000E3
:1002900001120100020000000842530200010001A7
:1002A00002000105010902A10185020901A1000561
:1002B0000919012908150025019508750181020514
:1002C00001093009311581257F95027508810609DC
:1002D000381581257F950175088106050C0A3802BD
:1002E0001581257F950175088106C0C0050109802B
:1002F000A101850319012AB700150126B700950150
:1003000075108100C0050C0901A101850419012A9D
:10031000A002150126A002950175108100C00501FB
:100320000906A101050719E029E71500250195082F
:10033000750181029501750881010507190029FFE2
:10034000150026FF0095067508810005081901298A
:1003500005950575019102950175039101C0112460
:100360001FBECFEFDAE0DEBFCDBF04B603FE18C07C
:100370008091940290919502A0919602B09197027B
:100380008730904BA740B04B59F4109294021092D2
:1003900095021092960210929702E0E0F8E3099518
:1003A00011E0A0E0B1E0ECE9F1E402C005900D92AB
:1003B000A03AB107D9F722E0A0EAB1E001C01D924E
:1003C000A439B207E1F70E949B120C94CC200C9444
:1003D0000000823038F4662311F08AEA01C089EA0D
:1003E0000E945D0481E0089581E0089581E0089510
:1003F0000C94F60108950C94FA011F93CF93DF93A8
:1004000000D000D01F92CDB7DEB749835A836B83EB
:100410003091A30189819A81311114C0662359F06A
:10042000222349F00E94B608182F682F89819A81EB
:100430000E945F0803C00E948A08182F69817A8190
:10044000812F04C00E94B60869817A810F900F90B5
:100450000F900F900F90DF91CF911F910C94061089
:10046000FC01262F408151816281738184810C942B
:10047000FD0181E00895CF93DF93EC0160E00E94DD
:100480003002BE01DF91CF910C94FB010C944C1112
:100490000C94481108950E9409070E944A022FEF08
:1004A00084E39CE0215080409040E1F700C00000D0
:1004B0000C945F190F931F93CF93DF938C0161E02E
:1004C0000E943002EC01B8010E94F8018823F1F18A
:1004D000B801CE010E947C178823C1F1B801CE017A
:1004E0000E943115882391F1B801CE010E94D816DF
:1004F000882361F1F8018281882309F1CB358DE5EC
:10050000D807C1F050F4C115FCE5DF0781F0CF3DFD
:10051000DC45A9F40E94ED0D19C0CC35EDE5DE07F0
:1005200061F0CD35DD4559F40E94300D08C00E94C0
:100530004B020CC00E94390D02C00E943C0DC80144
:10054000DF91CF911F910F910C94F40180E0DF9126
:10055000CF911F910F9108950E9493180C94D2028D
:100560000E94D5020C94991808950C94B40281E06D
:100570000895CF93C82F0E94B702882329F0C0FFA7
:1005800002C0299A01C02998CF910895219A2998EB
:100590000895CF93C82F0E94B5028C2F0E94B902F4
:1005A000CF91089580E00C94C9020E94D8170C9452
:1005B000C9020E94D8179091A201891721F0809357
:1005C000A2010C94C9020895CF93DF93CDB7DEB793
:1005D0002B970FB6F894DEBF0FBECDBF4F83588761
:1005E00069877A878B8761110E947C0C9E012F5F3F
:1005F0003F4F86E0F90111928A95E9F785E0FE0107
:100600003796D90101900D928A95E1F789819A81F7
:100610004C815D81452B31F09F3F31F491E08F3F5C
:1006200019F403C091E001C090E090FF09C0498136
:100630005A816B817C818D819E810E949D0B05C0BA
:10064000C9010E9439028111F2CF2B960FB6F8949E
:10065000DEBF0FBECDBFDF91CF910895FC01808139
:1006600091810E94F8080895CF93882309F4A4C0CB
:10067000C82F8238C1F40E94D81781FD9DC069E35C
:1006800080910201909103010E946B180E949E0CC0
:100690002FEF81EE94E0215080409040E1F700C0C0
:1006A000000069E319C0833801F50E94D81780FD66
:1006B00083C063E580910201909103010E946B1851
:1006C0000E949E0C2FEF81EE94E0215080409040DC
:1006D000E1F700C0000063E5809102019091030101
:1006E0000E946D18CF910C949E0C8438C1F40E9426
:1006F000D81782FD61C067E48091020190910301E7
:100700000E946B180E949E0C2FEF81EE94E0215006
:1007100080409040E1F700C0000067E4DDCF8CEF3F
:100720008C0F813AD0F46C2F8091020190910301DB
:100730000E943518882349F06C2F80910201909116
:1007400003010E946D180E949E0C6C2F8091020183
:10075000909103010E946B18C5CF80E28C0F883006
:1007600048F4C77081E001C0880FCA95EAF70E947B
:100770005F0CB8CFEBE5EC0FE33040F4F0E0E95B61
:10078000FE4F808190E0CF910C94FD17E8E5EC0FCF
:10079000E73150F4F0E0EE0FFF1FE75EFE4F80817F
:1007A0009181CF910C941318CD3E30F08C2F0E9484
:1007B0002013CF910C94F213CF910895882309F45C
:1007C00064C0823879F40E94D81781FF5EC069E363
:1007D00080910201909103010E946B180E949E0C6F
:1007E00069E310C08338B1F40E94D81780FF4DC070
:1007F00063E580910201909103010E946B180E94B1
:100800009E0C63E580910201909103010E946D1896
:100810000C949E0C843879F40E94D81782FF35C05E
:1008200067E480910201909103010E946B180E947D
:100830009E0C67E4E7CF9CEF980F913A10F4682F75
:10084000E1CF90E2980F983050F4877091E001C0AA
:10085000990F8A95EAF7892F0E94650CD9CF9BE5FD
:10086000980F933020F480E090E00C94FD1798E509
:10087000980F973120F480E090E00C9413188D3E8F
:1008800020F00E947B130C94F21308951F93CF93D2
:10089000DF93182FEB010E943403209741F08FE97A
:1008A0009FE00197F1F700C000002197F6CF812F5C
:1008B000DF91CF911F910C94DE03893319F060E032
:1008C00070E002C060E570E00C944604882321F0DB
:1008D0000E945F0C0C949E0C0895882321F00E94C6
:1008E000650C0C949E0C0895CF92DF92EF92FF92CC
:1008F0000F931F93CF93DF937C01D62FC72FFC015B
:100900001281058102950F700E94550C8823B9F061
:100910001123A9F08C2F807F803421F080E28D0F8D
:10092000883068F080916E0282FD09C082E00E94EA
:10093000FE0C0E94550C91E0D82ED92601C0D12C76
:10094000CC2EC2948FE0C8228C2D90E08C30910583
:1009500008F0CFC1FC01EA5AFF4F0C9463208C2FA2
:10096000807FCF70882311F0C295C07F112399F04A
:10097000CC2309F4AAC180E28D0F883010F0D11188
:1009800004C08C2F0E945F0C03C08C2F0E946F0C40
:100990000E949E0C9AC18D2F0E94DE03CC2309F485
:1009A000A8C180E28D0F883038F1DD2329F18C2F2A
:1009B0000E94750C24C08C2F807FCF70803211F084
:1009C000C295C07FDD2319F0D130A1F13DC08091E7
:1009D0006E0282FF17C0112349F0CC2329F08C2F1F
:1009E0000E945F0C0E949E0C80E070C180E00E941B
:1009F000DE03CC2309F47DC18C2F0E94650C0E947C
:100A00009E0C77C1112371F0002341F0013031F4C5
:100A10000E947F0C8C2B0E94870C6BC10E947F0C64
:100A20008C2B1DC0002319F0013009F462C10E9413
:100A3000940C25C0112321F0063008F05AC10EC0D5
:100A4000053008F056C11BC0112361F0002331F0BE
:100A5000F701858180FF39C18F7085838C2F0E94BB
:100A6000660447C1002359F0D93309F03FC1FFEFB5
:100A700007EE13E0F15000401040E1F735C18C2F34
:100A80000E946D0436C18C2F86958695837019F06F
:100A9000813061F02EC1112321F08D2F9C2F937096
:100AA00002C080E090E00E94FD172BC1112321F0CD
:100AB0008D2F9C2F937002C080E090E00E9413184D
:100AC00020C18D2F112319F00E94201302C00E9413
:100AD0007B130E94F21315C18C2F837009F047C05D
:100AE00011110BC12D2F229526952770220F220F51
:100AF0006D2F6F70862F90E0A0E0B0E0022E04C052
:100B0000880F991FAA1FBB1F0A94D2F7D4FF10C0E9
:100B10004FE050E060E070E004C0440F551F661FD6
:100B2000771F2A95D2F7409550956095709503C030
:100B300040E050E0BA01C695C695C3708A019B019A
:100B4000082B192B2A2B3B2BC901B801C23049F0C5
:100B500058F4C13019F00E947507CFC00E94630796
:100B6000CCC00E948707C9C00E946107C6C011237C
:100B700019F08C2F817001C08695882309F4BDC0BF
:100B80002D2F229526952770220F220F6D2F6F7023
:100B9000862F90E0A0E0B0E0022E04C0880F991FDD
:100BA000AA1FBB1F0A94D2F7D4FF10C04FE050E039
:100BB00060E070E004C0440F551F661F771F2A9540
:100BC000D2F7409550956095709503C040E050E095
:100BD000BA01C695C695C3708A019B01082B192BD3
:100BE0002A2B3B2BC901B801C23049F058F4C1305F
:100BF00019F00E943A0881C00E9428087EC00E9415
:100C00004C087BC00E949B0778C0CF70112339F03D
:100C10008C2F0E94C1078D2F0E9466046EC08D2FFD
:100C20000E946D048C2F0E94E20767C0D23F21F121
:100C300028F4D03F41F0D13FC1F043C0D33F19F178
:100C4000D43F79F03EC0112341F0053008F051C087
:100C50008C2F8F710E9407084CC0063008F049C0E5
:100C6000F7CF80916E0282FF18C0112339F08C2FCC
:100C70008F710E94C1073DC01123C9F38C2F8F7162
:100C80000E94E20736C0112329F08C2F8F710E9439
:100C9000AC072FC00E94A7072CC0112349F0CF71C9
:100CA0008C2F0E94C10763E08C2F0E94E30C21C0AF
:100CB00081E00E94FE0C0230E0F082E00E94FE0C17
:100CC00018C0112331F0002391F28D2F0E943403BC
:100CD00010C0002399F2D93349F41FEF27EE33E017
:100CE000115020403040E1F700C000008D2F0E94DD
:100CF000DE0388EF8C0D843020F40E94D8170E9408
:100D0000C902DD20C9F00E94510C80FD15C0F70119
:100D100012820E944B0C0E94C107C7010E94BD06AF
:100D20000E944B0CDF91CF911F910F91FF90EF909C
:100D3000DF90CF900C94E207DF91CF911F910F913C
:100D4000FF90EF90DF90CF9008950F931F93CF9374
:100D5000DF93EC01688179818A810E9403098C010B
:100D60000E945E080E944F07B801CE010E947404E1
:100D7000DF91CF911F910F910895CF93DF93EC01F5
:100D8000988189812B813C81232B31F08F3F31F475
:100D900081E09F3F19F403C081E001C080E080FD45
:100DA0001DC0CE010E945A02811110C00E94550C34
:100DB0008823A1F08A81882389F080916E0282FDC8
:100DC0000DC082E0DF91CF910C94FE0CCE010E9409
:100DD000A506CE01DF91CF910C943B02DF91CF911C
:100DE000089580E090E00E94FD1780E090E00E946E
:100DF00013180E947C0C0E949E0C0E9423150C94D8
:100E0000F21380910201909103010E946F180C94DB
:100E1000F1060E946C0C0C94010792959F7096301D
:100E200079F010F4925001C09A50923068F4803FEB
:100E300069F018F4883E40F409C0843F29F406C0E4
:100E4000883E20F0813F11F080E0089581E0089510
:100E5000FC01808191810E94F8080E940D0708958D
:100E6000CF93DF9300D000D01F92CDB7DEB70F90A5
:100E70000F900F900F900F90DF91CF910895CF9327
:100E8000DF9300D000D000D0CDB7DEB726960FB6E6
:100E9000F894DEBF0FBECDBFDF91CF9108950895C6
:100EA00008950C9450070C9451070E9453076093C7
:100EB000DA017093DB018093DC019093DD010C94E7
:100EC000F1060C9455070F931F930091DA011091CE
:100ED000DB012091DC013091DD01602B712B822B35
:100EE000932B1F910F910C9455070F931F93009113
:100EF000DA011091DB012091DC013091DD016023EA
:100F00007123822393231F910F910C9455070F9304
:100F10001F930091DA011091DB012091DC013091E7
:100F2000DD0160277127822793271F910F910C9471
:100F300055070C9450070E9499076093D60170934F
:100F4000D7018093D8019093D9010C94F10660E009
:100F500070E0CB010C949B070F931F9341E050E08E
:100F600060E070E08A019B0104C0000F111F221F86
:100F7000331F8A95D2F7C901B8011F910F910C94C4
:100F80009B070F931F9341E050E060E070E004C0C6
:100F9000440F551F661F771F8A95D2F78091D6019F
:100FA0009091D701A091D801B091D9018A019B01FC
:100FB000082B192B2A2B3B2BC901B8011F910F912C
:100FC0000C949B070F931F9341E050E060E070E0AA
:100FD00004C0440F551F661F771F8A95D2F74095AE
:100FE0005095609570958091D6019091D701A09110
:100FF000D801B091D9018A019B01082319232A2322
:101000003B23C901B8011F910F910C949B070F93CB
:101010001F9341E050E060E070E004C0440F551FB2
:10102000661F771F8A95D2F78091D6019091D701DC
:10103000A091D801B091D9018A019B0108271927F5
:101040002A273B27C901B8011F910F910C949B07D8
:101050000F931F930091D6011091D7012091D801D1
:101060003091D901602B712B822B932B1F910F9103
:101070000C949B070F931F930091D6011091D701F9
:101080002091D8013091D9016023712382239323C9
:101090001F910F910C949B070F931F930091D60102
:1010A0001091D7012091D8013091D9016027712783
:1010B000822793271F910F910C949B0708952FE08F
:1010C000929F800D1124E82FE695E695E6958770AE
:1010D00051E001C0550F8A95EAF785E0E89FF001DD
:1010E0001124EC55FE4F20E030E070E04081CB0150
:1010F000022E02C0969587950A94E2F78170819539
:1011000084278523842781932F5F3F4F2530310526
:1011100069F708952FE0929F800D1124682F66953E
:1011200066956695982F977085E0689FB0011124A9
:1011300040E050E080E0FB01E40FF51FEC55FE4F6E
:10114000208130E0092E02C0369527950A94E2F7F7
:1011500021703327042E01C0220F0A94EAF7822B54
:101160004F5F5F4F4530510531F70895BF92CF92E1
:10117000DF92EF92FF920F931F93CF93DF938C0137
:10118000C090D601D090D701E090D801F090D9015D
:101190008091DA019091DB01A091DC01B091DD0139
:1011A000C82AD92AEA2AFB2ACFE1D0E0D701C60112
:1011B0000C2E04C0B695A795979587950A94D2F7FB
:1011C00080FD04C0219790F7B12C07C0BC2EB80158
:1011D0008C2F0E9419100197A9F38B2DDF91CF91CD
:1011E0001F910F91FF90EF90DF90CF90BF900895E7
:1011F000CF93DF93EC010E94B608BE010E94191044
:10120000DF91CF9108951F93CF93DF93EB019091DE
:10121000A301992321F0CB010E94F80813C0882371
:1012200049F0CB010E94B608182F682FCE010E940A
:101230005F0804C0CB010E948A08182FBE01812FCD
:101240000E941910DF91CF911F9108951F93CF93A2
:10125000DF93C091DE0116E08091DF01C81799F09D
:10126000D0E01C9FF0011D9FF00D1124E052FE4FB5
:101270004081518162817381848195810E943F0701
:101280002196C770E9CFDF91CF911F9108954091CA
:10129000100250911102609112027091130280911C
:1012A0001402909115020C943F07EF92FF920F9356
:1012B0001F93CF93DF938091150282958F7009F071
:1012C00065C080911202882309F460C08091DE011C
:1012D000F090DF0110911002009111026091130251
:1012E0007091140291E01F3F09F090E0C09100015D
:1012F000D0910101292F96E0E92E8F1509F446C0FF
:101300006115710521F00F3F21F030E003C031E09D
:1013100001C0322F90E030FD36C0E89EF001E99E1A
:10132000F00D1124DF01A052BE4F11963C91119790
:10133000301329C03C91311326C012963C9112976C
:10134000311121C013964D915C911497461B570B98
:101350004C175D07C0F4809115028F7080618093F7
:101360001502EB51FE4F80818F708061808380E198
:1013700092E00E94BD06DF91CF911F910F91FF90E7
:10138000EF900C94260901968770B7CFDF91CF912B
:101390001F910F91FF90EF9008959F92AF92BF928F
:1013A000CF92DF92EF92FF920F931F93CF93DF9331
:1013B000CDB7DEB761970FB6F894DEBF0FBECDBFD5
:1013C0008C0185E0F801DE011D9601900D928A9551
:1013D000E1F7D8011296EC9090911002E091110281
:1013E00020911302309114022115310531F0EF3FA5
:1013F00031F481E09F3F19F403C081E001C080E037
:10140000B82FB1709B2E80FD47C1D8014C91119629
:101410005C9111971396AD90BC90149780E1C82E03
:1014200082E0D82EF0901202B501621B730B20915E
:10143000000130910101FF2009F4D9C0809115020B
:101440006217730708F095C0282F207F09F052C05B
:101450005E1313C0491311C0FE2CE1100EC08F7033
:101460008061809315020E944709C6010E94BD0653
:1014700080911502F80185834DC1AB2831F05F3FA3
:1014800031F481E04F3F19F403C081E001C080E0F6
:1014900080FD03C081E08E2502C080E090E0F82F3F
:1014A000F170FF2E80FF1CC08091DE012091DF01D2
:1014B00036E0821709F40BC190E0389FF001399FA4
:1014C000F00D1124E052FE4F6181561306C0608179
:1014D000461303C06281E61203C001968770E9CF0C
:1014E000FE2CEE2009F416C18091150281608093D4
:1014F000150254C05E1306C0491304C0E11002C0B7
:10150000F80199C0C8010E942807882361F1EE20E4
:1015100051F120911502822F82958F7090E00297F1
:1015200074F0809110029091110298878F83198630
:10153000BB86AA862C87CE0107960E94BD0686E050
:10154000F801A0E1B2E001900D928A95E1F70E94C6
:1015500055090E9447090AC05E1711F1C8010E948F
:10156000280781112CC0C8010E94BD06FF24F394F6
:10157000D1C0282F207F81F77A2DB98AA88A6E2DB5
:1015800089890E94300780E192E00E94BD0686E0D2
:10159000D6011D928A95E9F70E944709F12CBAC03D
:1015A0004913DCCFE110DACFF8018583C8010E942E
:1015B000BD0686E0D6011D928A95E9F7ABC0EE2004
:1015C00091F220911502822F82958F7090E0029700
:1015D0000CF4B5CF80911002909111029A83898307
:1015E0001B82BD82AC822E83CE010196A6CF6217EC
:1015F000730708F044C0FE2CEE2009F4B4CF5E134C
:1016000030C049132EC02091150220FD21C0822F29
:1016100082958F70482F50E041155105C9F0F801AF
:1016200025834F30510541F08F5F982F9295907F21
:10163000822F8F70892B8583C8010E94BD0686E0AA
:10164000F801A0E1B2E001900D928A95E1F73CC06B
:1016500086E0F801A0E1B2E001900D928A95E1F7F1
:1016600059C0C8010E942807811169CF80911502D5
:10167000816080931502C8010E94BD064BC07A2D7F
:10168000B98AA88A6E2D89890E94300786E0D60122
:101690001D928A95E9F718C0EE2009F464CFC801BD
:1016A0000E942807F82E882309F45DCF86E0F80110
:1016B000A0E1B2E001900D928A95E1F780E192E01D
:1016C0000E942E030E9455090E94470923C04D879E
:1016D0005E878D859E850E94F808292F22952F70A0
:1016E000223028F49F7039F0811105C00BC02430DE
:1016F00028F49F7049F4805E883020F0C8010E9471
:10170000BD069F2CF92C06C0D80115969C91907FA0
:1017100091F7F8CF8F2D61960FB6F894DEBF0FBE0C
:10172000CDBFDF91CF911F910F91FF90EF90DF9090
:10173000CF90BF90AF909F9008951F93CF93DF936A
:10174000CDB7DEB72C970FB6F894DEBF0FBECDBF76
:101750004F83588769877A878B879C87CE01079646
:101760000E94CD098823D1F09F8188852A853B85F9
:10177000232B31F08F3F31F481E09F3F19F403C0F8
:1017800081E001C080E080FD47C04F8158856985B8
:101790007A858B859C850E943F073EC086E0FE01CE
:1017A0003796DE01119601900D928A95E1F7FF813F
:1017B000E8856A857B856115710531F0EF3F31F46D
:1017C00081E0FF3F19F403C081E001C080E080FDAB
:1017D00023C02091DF0130E0C9010196877099276D
:1017E0004091DE0150E084179507F1F1F983EA8317
:1017F0007D836C8396E0929FD001939FB00D11245E
:10180000A052BE4FFE01319601900D929A95E1F7DC
:101810008093DF010E94260916E08091DE019091FD
:10182000DF01891771F1189FC001112480529E4F6A
:101830000E94CD09882329F1E091DE011E9FF0016D
:101840001124E052FE4F4081518162817381848175
:1018500095810E943F078091DE0190E0019687709C
:1018600099278093DE01D9CF0E9409071092DF01EA
:101870001092DE01E0E1F2E086E0DF011D928A9540
:10188000E9F72C960FB6F894DEBF0FBECDBFDF91FF
:10189000CF911F91089580911E028595859585951C
:1018A000089580911E028770089590911E0297708E
:1018B00081E009F480E008958091290208959091D3
:1018C0002902892B809329020895809590912902FD
:1018D00089238093290208951092290208959091F6
:1018E0002802892B809328020895809590912802E0
:1018F00089238093280208951092280208958091E8
:101900001F02089508950C94820C0C94830C9091FE
:101910006E0292FD08C090911F02981721F08093EB
:101920001F020C94850C089580911F02882329F0D2
:1019300010921F0280E00C94850C0895CF93DF93E2
:10194000E0910201F0910301809129028083E091EE
:101950000201F0910301908180912802892B8083FC
:1019600080911F02882381F0E0910201F091030130
:101970009081892B808380910201909103010E94C4
:10198000291881110E94940CC0910201D091030189
:1019900048E050E066E172E0CE010E947D20892B94
:1019A00069F088E0FE01A6E1B2E001900D928A950F
:1019B000E1F7CE01DF91CF910C94E417DF91CF9145
:1019C00008950C94820C90916E0292FD10C098E0E4
:1019D000899F90011124262B20931E020E94C1078B
:1019E00080911E028595859585950C94E10C0C944B
:1019F000C10710921E0280E00C94E10C20911E029F
:101A00008095822380931E02982F977099F430E07E
:101A1000482F082E000C550B2417350759F09091CC
:101A20006E0292FD07C08595859585950E94E20717
:101A30000C94F90C089590916E0292FB222720F9E4
:101A4000281769F080FB92F990936E0280916D02E5
:101A500090916E020E94690D82E00C94FE0C089534
:101A600080916E0282FB882780F991E089270C948F
:101A70001B0D81E00C941B0D80E00C941B0D6FEF8F
:101A80007FEF80E090E00C94B62080E090E00E9430
:101A9000922021E0893E9E4F09F020E0822F089598
:101AA00082E090E00C948A2083E090E00C948A20FD
:101AB000CF9384E090E00E948A20C82F82E290E0D9
:101AC0000E948A202C2F30E0A901582BCA01CF9107
:101AD0000895CF93C92F682F84E090E00E9498204A
:101AE0006C2F82E290E0CF910C949820AB01BC0166
:101AF0008FE090E00C94AA20AB01BC0183E190E060
:101B00000C94AA2060E070E0CB010C947C0D60E0A6
:101B100070E0CB010E94760D0C94820D69EE7EEF91
:101B200080E090E00E94B62060E082E090E00E94B9
:101B3000982060E083E090E00E9498201092DA0103
:101B40001092DB011092DC011092DD0160E084E074
:101B500090E00E94982060E082E290E00E9498204D
:101B600060E085E090E00E94982060E086E090E0F0
:101B70000E9498206FEF87E090E00E94982040E05C
:101B800050E0BA0188E090E00E94AA2060E08DE079
:101B900090E00E94982040E050E0BA0188E190E097
:101BA0000E94AA2060E087E190E00E94982040E037
:101BB00050E0BA018CE190E00E94AA2060E070E061
:101BC00080E290E00E94B62040E050E0BA0188E157
:101BD00090E00E94AA200C94870D0C948E0D682F23
:101BE0008EE090E00C9498200E941E1960933C02B5
:101BF00070933D0280933E0290933F0260933802BF
:101C00007093390280933A0290933B0208950E94A8
:101C10001E1960933C0270933D0280933E029093A4
:101C20003F026093340270933502809336029093A2
:101C30003702089585B7806885BF85B7806885BFFE
:101C4000089581E008950C94210E08950C94250EBA
:101C50000C94250E0C94280E0C94250E0C942C0E2E
:101C60000C94250E0E941A0E85EF90E10E94CE176B
:101C70000E94300E0C942E0E0E94260E0C94250EFF
:101C80000E940F110C94C6020E9409190E94F411BF
:101C90000E94400E0E9482160C942A0E5F926F9250
:101CA0007F928F929F92AF92BF92CF92DF92EF92EC
:101CB000FF920F931F93CF93DF93CDB7DEB72A9791
:101CC0000FB6F894DEBF0FBECDBF0E940912C82E1A
:101CD00081110E94F40D3AE2832E32E0932E00E04F
:101CE00010E0502E802F0E9433115C01F4016190AE
:101CF00071904F016826792661147104B1F40F5F69
:101D00001F4F0530110569F78FEF89838A831B8286
:101D10000E9412198160782F9D838C8349815A819A
:101D20006B818D810E94E4023AC08091400281FD66
:101D30000E943C11D12CEE24E394F12CC3018E219E
:101D40009F21892B29F10E94230E8823A9F0DE828E
:101D50005F82AE20BF2081E0AB2809F480E0888755
:101D60000E9412198160782F9A8789874E815F813E
:101D700068858A850E94E402000F111FF801E65D64
:101D8000FD4F80819181E826F926F182E08207C02B
:101D9000D394EE0CFF1CFFE0DF12D0CFB0CF81E078
:101DA000C11001C080E02A960FB6F894DEBF0FBEC6
:101DB000CDBFDF91CF911F910F91FF90EF90DF90FA
:101DC000CF90BF90AF909F908F907F906F905F90DB
:101DD00008950E944E0E0E94951681110E94070ED2
:101DE0000E9410140C94D902CF93DF930E941E100E
:101DF000EC01811521E5920708F045C0811530E519
:101E0000930708F094C0883E910528F5803E91051F
:101E100008F0F8C0883A910570F4853A910508F009
:101E20007CC08130910509F475C008F4E8C00497BE
:101E300008F0E8C0E4C08F3B910508F0E0C0C85A44
:101E4000D0E0CC0FDD1FC65BDE4F0990D881C02DDE
:101E5000CE019464D8C0811540E2940758F48115EE
:101E600051E0950708F0CEC08D3E910508F4C7C03B
:101E70009065C9C0C11580E4D80708F4C0C0DF7000
:101E8000CE01906AC0C0811525E59207A8F481159E
:101E900034E5930708F095C0811543E5940708F0F1
:101EA0007BC0811552E5950708F061C0D82FCC277B
:101EB000CE01816F906AA7C0C11589E5D807A0F44B
:101EC000C11528E5D20708F082C0C11536E5D30751
:101ED00008F095C08C2F0E94B2108F7190E0D82F1F
:101EE000CC27CE0190628FC0C1154AE5D40708F413
:101EF00074C0CE0190568115904208F080C08D2F9D
:101F00008F710E94B210DD27D0628F71AE01582B05
:101F1000CA0179C081E090E076C0C55AD0E0C858C7
:101F2000DE4F8881C82FD0E0CE0190646CC074E091
:101F3000969587957A95E1F7282F23703C2F33707B
:101F400081E090E002C0880F991F3A95E2F79C6803
:101F5000AC01522B9A019C2F9F709695969550E25A
:101F6000959FE0011124C9018C2B9D2B4CC08370DF
:101F7000992721E030E002C0220F331F8A95E2F753
:101F80009C2F9695969580E2989FE0011124C22B94
:101F9000D32BCE019C6837C08370992721E030E0B5
:101FA00002C0220F331F8A95E2F79C2F96959695D3
:101FB00040E2949FE0011124C22BD32BCE019A68FA
:101FC00022C0D82FCC27CE01846F906A1CC0DC2F92
:101FD000CC27CE01806F906A16C08C2F8F700E9424
:101FE000B21094E0D695C7959A95E1F7CF70D0E0FE
:101FF000DC2FCC27D0699E01282BC90104C080E0CA
:1020000090E001C0CE01DF91CF9108952BE4829F33
:10201000C0011124FC012FE0729FE00DF11D11247D
:10202000E60FF11DEE0FFF1FE852FF4F85919491CF
:1020300008950E9406100E94F40E089582389105BA
:1020400069F1B0F48133910509F46DC048F4893227
:10205000910509F463C08A32910509F469C00895B5
:102060008533910509F455C089339105B9F0089578
:10207000833E910569F138F4803E9105B1F0823ECE
:10208000910509F10895863E9105A9F1873E9105D4
:10209000B9F1843E910509F064C023C020916D021E
:1020A00020FD4FC021FD4DC0089580916D0280FD3F
:1020B00044C080916E0280FF44C080916D0284FD17
:1020C00042C083EE4DC080916D0282FF38C0F5CFD3
:1020D00080916D0282FD33C080916E0280FD31C01F
:1020E000ECCF80916E0281FF32C080916D0284FD41
:1020F0002AC087EE35C080916D0283FF26C0F5CFE0
:1021000080916D0283FD21C080916E0281FD1FC010
:10211000ECCF80916D0285FD1CC01DC080916D02C9
:1021200085FD19C016C080916D0286FD16C017C0CE
:1021300080916D0286FD13C010C089E311C082EE4C
:102140000FC080EE0DC080E00BC086EE09C084EEAB
:1021500007C089E205C085E303C08AE201C081E3CC
:1021600090E0089590916D0292FF0DC0282F287184
:10217000283019F4877F846006C0282F247124300A
:1021800011F48B7F886093FF0DC0282F28712831B0
:1021900019F4877E846106C0282F2471243111F43C
:1021A0008B7E886120916E0220FF0DC0382F387120
:1021B000383019F4877F816006C0382F3171313093
:1021C00011F48E7F886021FF0DC0282F28712831DF
:1021D00019F4877E816106C0282F2171213111F405
:1021E0008E7E886194FD877E089580E008950C942A
:1021F0003F0D0E9409128FE39CE90197F1F700C09F
:1022000000000E94091281E00E94331180FF04C087
:102210000E94F7100C945F1908950C94F9100E9415
:10222000450D811102C00E94ED0D0E94500D80935A
:1022300040020E94580D90936E0280936D020E949E
:102240000D110E94540D682F70E080E090E00E9414
:1022500061076091D6017091D7018091D80190916A
:10226000D9010C949907E82FF0E0EE0FFF1FE75813
:10227000FD4F808191810895089580EA8A95F1F754
:10228000089500C008950C943D1108950C944511D3
:102290000C9446110C9445110C944A11F894E82FB3
:1022A000E295EF70F0E031A1282F2F7081E090E0EF
:1022B00001C0880F2A95EAF7982F9095932391A350
:1022C00092A1892B82A3789408950F931F93CF93A3
:1022D000DF93CAE8D1E089918F3F11F00E944E113F
:1022E00081E0CF38D807B9F7CBE7D1E00AE811E0B1
:1022F00089918F3F11F00E944E110C171D07C1F7F5
:10230000DF91CF911F910F910895BF92CF92DF92ED
:10231000EF92FF920F931F93CF93DF938C01C62F01
:10232000D0E0CE0186579E4F6C01FC0190819F3F0B
:1023300009F450C0B62EF894E92FE295EF70F0E062
:1023400081A19F7021E030E001C0220F9A95EAF749
:10235000822B81A382A12095282322A378940E9416
:102360004111EBE7F1E04AE851E021E030E0E12CF7
:10237000F12C61916F3F89F0A62FA295AF70B0E06C
:1023800090968C9190E06F7002C0959587956A95B4
:10239000E2F780FD02C0C90102C080E090E0E82AB7
:1023A000F92A220F331F4E175F0719F7F6018081B4
:1023B0008F3F11F00E944E1161E0E114F10409F425
:1023C00060E08B2D0E944311CC0FDD1FC00FD11F89
:1023D000F982E882DF91CF911F910F91FF90EF90EA
:1023E000DF90CF90BF9008950E9465118AE0E9E7E1
:1023F000F2E0DF01982F1D929A95E9F7EFE6F2E0FF
:10240000DF011D928A95E9F785E00E9454120C9431
:102410004602FF920F931F93CF93DF93CDB7DEB7A2
:102420002A970FB6F894DEBF0FBECDBF8E010F5FA7
:102430001F4F8AE0F80111928A95E9F7F12C6F2D70
:10244000C8010E948511F394F5E0FF12F8CF4AE02D
:1024500050E0B8018FE692E00E947D20FF24F394C3
:10246000009709F4F12C892B41F08AE0F801AFE6DE
:10247000B2E001900D928A95E1F72F2D45E069E7D2
:1024800072E08FE692E00E9455120E9448028F2D62
:102490002A960FB6F894DEBF0FBECDBFDF91CF9165
:1024A0001F910F91FF9008950895FF920F931F932E
:1024B000CF93DF93F82E092F162FD72FC42F222367
:1024C00049F081E0809343020E94121990934202E6
:1024D00080934102809143028823D9F08091410288
:1024E000909142020E942A19059798F0EF2DF02F43
:1024F000A12FBD2F80E090E04C2F50E0841795076E
:1025000034F4219131912D933D930196F7CF1092A0
:102510004302DF91CF911F910F91FF9008950E9488
:10252000151B0E94440E0C94211B0E94251B0E9427
:10253000E90E0C943F1B0E94B0180E94FC1A0E94E6
:10254000320E0E948F120E9495120E943C0EFBCF09
:1025500080914A0280FF06C06091090170E0660F19
:10256000771F26C081FF04C06091090184E005C087
:1025700082FF07C06091090188E0689FB0011124C3
:1025800017C0909149029923D1F0609108019617E4
:1025900088F72091090188E0289F90011124929FDB
:1025A000A001939F500D112470E0CA010E944F209A
:1025B0006038710540F46115710519F406C068E0D2
:1025C00070E0862F08958FE7089581E00895809147
:1025D0004A0280FF08C06091050170E0759567951B
:1025E0007595679521C081FF06C06091050170E077
:1025F0007595679519C082FF04C06091050170E070
:1026000010C090914802992399F0609104019617A7
:10261000A0F780910501899FC001112470E00E94FC
:102620004F206038710540F46115710519F406C03A
:1026300061E070E0862F08958FE7089581E00895A6
:102640008D3E21F40E94A812819504C08E3E29F48B
:102650000E94A81280934E0208958F3E21F40E949A
:10266000A812819504C0803F29F40E94A81280938B
:102670004D020895893F19F40E94E71205C08A3F70
:1026800031F40E94E712819580934F0208958B3FA9
:1026900021F40E94E712819504C08C3F29F40E9426
:1026A000E7128093500208959FE0980F983078F4D5
:1026B00021E030E0A90102C0440F551F9A95E2F7CE
:1026C000CA0190914C02892B80934C0208958D3F52
:1026D00021F480914A0281600BC08E3F21F48091E9
:1026E0004A02826005C08F3F29F480914A028460CB
:1026F00080934A0208958D3E39F490914E0297FFDF
:1027000035C010924E0259C08E3E29F490914E026F
:102710001916BCF32BC090914D028F3E29F497FF00
:1027200025C010924D0249C0803F19F41916CCF310
:102730001DC090914F02893F29F41916BCF41092E4
:102740004F023BC08A3F19F497FF10C0F8CF8B3F70
:1027500039F49091500297FF09C0109250022DC099
:102760008C3F21F4909150021916BCF39FE0980F12
:10277000983080F421E030E0A90102C0440F551FD9
:102780009A95E2F7CA01809590914C028923809333
:102790004C0213C08D3F21F480914A028E7F0BC002
:1027A0008E3F21F480914A028D7F05C08F3F29F42E
:1027B00080914A028B7F80934A0280914D02811161
:1027C00006C080914E02811102C010924902809190
:1027D0004F02811106C080915002811102C01092F7
:1027E000480208950E94121920914D02211104C03F
:1027F00020914E02222321F09093470280934602BB
:1028000020914F02211104C020915002222321F077
:1028100090934502809344028BE492E00C94EF176E
:10282000EF92FF920F931F93CF93DF9300D000D0CE
:1028300000D0CDB7DEB786E0EBE4F2E0DE01119622
:1028400001900D928A95E1F7E0904D02F0904E02D2
:1028500000914F021091500210924D0210924E02C0
:1028600010924F0210925002E11003C0FF2009F4B1
:102870005DC080914602909147020E942A19AC01E6
:1028800090914902992339F020910A0130E02417F0
:10289000350758F04BC020910B018AE0289F90012A
:1028A00011242417350718F041C09F3F19F09F5F8E
:1028B00090934902EE2061F00E94A8121E1414F0B9
:1028C0009FEF01C091E0989F902D112490934D02AD
:1028D000FF2061F00E94A8121F1414F09FEF01C0A6
:1028E00091E0989F902D112490934E0230914D02CB
:1028F0003323E1F020914E022223C1F045EB340353
:10290000C0011124992319F090934D0203C081E076
:1029100080934D0235EB2303C0011124992319F054
:1029200090934E0203C081E080934E02011103C0D8
:10293000112309F45DC080914402909145020E94E8
:102940002A19AC0190914802992339F0209106018F
:1029500030E02417350758F04BC0209107018AE07A
:10296000289F900111242417350718F041C09F3F7C
:1029700019F09F5F90934802002361F00E94E712D4
:10298000101614F09FEF01C091E0989F902D112434
:1029900090934F02112361F00E94E712111614F078
:1029A0009FEF01C091E0989F902D112490935002C9
:1029B00030914F023323E1F0209150022223C1F0E5
:1029C00045EB3403C0011124992319F090934F0271
:1029D00003C081E080934F0235EB2303C001112433
:1029E000992319F09093500203C081E08093500224
:1029F00080914D0281110BC080914E02811107C060
:102A000080914F02811103C08091500281110E9478
:102A1000F213EB82FC820D831E8386E0FE01319669
:102A2000ABE4B2E001900D928A95E1F726960FB6DD
:102A3000F894DEBF0FBECDBFDF91CF911F910F91F4
:102A4000FF90EF900895EBE4F2E086E0DF011D9245
:102A50008A95E9F7109249021092480210924A02B0
:102A60000895CF93DF93EC01FB018281882309F461
:102A70003CC1C430FDE5DF0760F4CB3F9CE5D907DE
:102A800088F49E0122503C452431310508F02EC1C6
:102A900009C0C236EDE5DE0729F0C63AFDE5DF07DD
:102AA00009F024C10E94580D90936E0280936D022C
:102AB000C1318CE5D80709F4C6C008F042C0C9305E
:102AC000ECE5DE0709F49BC000F5C5308CE5D807BE
:102AD00009F485C078F4C330ECE5DE0709F478C06A
:102AE00008F07AC0C230DC4509F0F5C080916D0273
:102AF0008160EFC0C7309CE5D90709F478C008F0C1
:102B00007AC080916D028061E4C0CD30FCE5DF07C2
:102B100009F487C058F4CB309CE5D90709F479C093
:102B200008F07BC080916D0288606FC0CF30FCE5FB
:102B3000DF0709F480C008F082C080916D02877FB2
:102B4000C8C0CE3F9CE5D90709F471C000F5C53176
:102B5000FCE5DF0709F485C068F4C3319CE5D907BB
:102B600009F475C008F095C00E94090780916D02B4
:102B70008F77AFC0CC3FFCE5DF07A9F108F054C068
:102B8000CB3FDC4509F0A7C080916E0240C0C23047
:102B9000EDE5DE0709F489C058F4C1158DE5D807C5
:102BA00009F45AC008F069C080916E0282602FC09B
:102BB000C236EDE5DE0709F47CC0C63AFDE5DF0765
:102BC00009F481C0C330DD4509F085C080E06EC0E6
:102BD00080916D0282607DC080916D0216C08091EF
:102BE0006D02886076C080916E0282604FC08091D5
:102BF0006D0280626EC080916D0280646AC00E9426
:102C0000090780916D02806864C0846062C0816041
:102C10003DC080916D028E7F5CC080916D028D7F82
:102C200058C080916D0216C080916E0218C08091CC
:102C30006E028D7F2BC080916D028F7E4AC0809185
:102C40006D028F7D46C080916D028F7B42C0809166
:102C50006D02877F8B7F3DC080916E028D7F8E7F5E
:102C600015C080916D0282FB222720F991E0922706
:102C700090FB82F990FB83F92CC080916E02982F13
:102C8000909591708E7F892B90FB81F980936E02D5
:102C900022C00E94090780916D0287FB222720F93C
:102CA00091E0922790FB87F914C081E00E94EF0D1C
:102CB00012C080916D0284FB222720F991E09227B7
:102CC00090FB84F906C080916D02982F909590FB3F
:102CD00080F980936D0280916D0290916E020E9446
:102CE000690D0E94090780E001C081E0DF91CF916A
:102CF00008958FE891E00197F1F700C00000089572
:102D00000C94E90123982B9A22982A9A0E9479160A
:102D100083B183FB882780F91A9902C090E001C033
:102D200092E0892B809353020895E0915302EE0FB5
:102D3000EE0FE093530243B143FB882780F990E004
:102D400043B142FB222720F930E042FF02C022E0DB
:102D500030E0822B932B8E2B809353028F70E82FC1
:102D6000F0E0E157FE4F908180915202890F8093ED
:102D7000520218165CF4809151028F5F80935102C9
:102D800060E080E00E94801681E001C080E09091C8
:102D9000520297FF0AC080915102815080935102E4
:102DA00061E080E00E94801681E010925202089556
:102DB000CF93DF9386319C4541F5EB010E945C0C7B
:102DC000982F8A812091020130910301882379F0A4
:102DD0009A7A81E009F480E080935402911102C054
:102DE00069E201C065E3C9010E946B180AC08091C5
:102DF0005402811102C069E201C065E3C9010E9469
:102E00006D180E949E0C80E001C081E0DF91CF919F
:102E100008950F931F93CF93DF93C42FD22FFC01FC
:102E200082818823C9F0409357020E94121990931F
:102E300056028093550280E28C0F883008F057C00C
:102E4000C77081E001C0880FCA95EAF7DF91CF9182
:102E50001F910F910C94660480915702481330C063
:102E600080915502909156020E942A19883C910542
:102E700038F510E21D0FCD17B9F080E28C0F8830C5
:102E800040F4C77081E001C0880FCA95EAF70E943C
:102E90006D04183028F581E09D2F977001C0880FD0
:102EA0009A95EAF70E946604802F0E945D0418300C
:102EB000F0F4D77081E001C0880FDA95EAF70AC014
:102EC00080E28C0F883098F4C77081E001C0880FD1
:102ED000CA95EAF7DF91CF911F910F910C946D0481
:102EE000802FDF91CF911F910F910C945D04DF91A2
:102EF000CF911F910F9108950F939C01CB01243F17
:102F00004CE5340731F188F4293DFCE53F07D9F061
:102F10002A3D4CE5340779F1283D3C45A9F506E208
:102F200021EE41EE68ED7CE52BC0263FFCE53F0736
:102F3000E1F0A8F0273F3C4539F507E225EE46EEE3
:102F400067EF7CE51DC007E225EE45EE69ED7CE507
:102F500017C006E221EE40EE64EF7CE511C007E207
:102F600025EE44EE65EF7CE50BC006E221EE42EE75
:102F700066EF7CE505C008E221E045EE6AED7CE500
:102F80000E94091780E008C0FC018281882319F0A3
:102F90001092570201C081E00F9108959093A10112
:102FA0008093A001089590935D0280935C02089540
:102FB000E0915C02F0915D02309721F00190F08188
:102FC000E02D099480E00895E0915C02F0915D02AB
:102FD000309721F00280F381E02D09940895E0916B
:102FE0005C02F0915D02309739F022E0DC012C9315
:102FF0000480F581E02D0994089520915A023091C2
:103000005B022817390771F090935B0280935A0294
:10301000E0915C02F0915D02309721F00680F7812B
:10302000E02D0994089520915802309159022817F3
:10303000390771F09093590280935802E0915C0235
:10304000F0915D02309721F00084F185E02D099424
:103050000895FC01329697E080E0915029F021918B
:103060002223D9F38F5FF9CF0895662349F0FC013D
:10307000329608962191621729F0E817F907D1F7DF
:1030800080E0089581E008959C01FC0132969FEF55
:1030900080E04191461789F09F3F19F4411101C02A
:1030A000982F8F5F8630A9F79F3F39F0F901E90F1C
:1030B000F11D97FDFA956283089508959C012A5F9A
:1030C0003F4FFC014281461301C0128201968217D4
:1030D0009307B9F708950C9444180C945E1802965F
:1030E00026E0FC0111922A95E9F7089508950C94C1
:1030F000761883E080935E020C947718811102C0E9
:1031000081E001C082E080935E020C9477180C94F9
:103110007E1881E080935E020C9477180C948918D5
:1031200008950C9490180C9491180C9490180C9489
:1031300090180C949018CF930E9497180E9409122F
:103140000E949518C0E08C2F0E943311892B29F41E
:10315000CF5FC530C1F780E001C081E0CF91089515
:1031600008951F920F920FB60F9211248F939F9381
:10317000AF93BF9380915F02811113C0809183024E
:1031800090918402A0918502B09186024196A11D82
:10319000B11D8093830290938402A0938502B09323
:1031A0008602BF91AF919F918F910F900FBE0F90AC
:1031B0001F90189580918B02843031F10E94AC02EF
:1031C00010925F0220E488E190E00FB6F894A89591
:1031D000809360000FBE2093600083B7817F84607E
:1031E00083BF83B7816083BF7894889583B78E7FD0
:1031F00083BF0FB6F894A895809160008861809392
:103200006000109260000FBE08950E9409070C94A0
:10321000B00282E084BD93E095BD9AEF97BD8093A4
:103220006E0008952FB7F8948091830290918402E4
:10323000A0918502B09186022FBF08952FB7F89410
:103240006091830270918402809185029091860240
:103250002FBF08959C014FB7F894809183029091FD
:103260008402A0918502B09186024FBF821B930B0E
:10327000089578941F920F920FB60F9211248F9396
:103280009F93AF93BF938091830290918402A0910A
:103290008502B09186020196A11DB11D8093830223
:1032A00090938402A0938502B0938602BF91AF9160
:1032B0009F918F910F900FBE0F901F90189581E0F6
:1032C0008093E00080E28093D8001092C9008FE1E3
:1032D0009EE40197F1F700C0000087E090EBDC016D
:1032E0008093940290939502A0939602B0939702D4
:1032F0009CE088E10FB6F894A895809360000FBE1B
:1033000090936000FFCF80916B020895089522E0B2
:103310002093E9002FEF3091E800215035FD06C0E1
:1033200035ED3A95F1F700002111F5CF2091E80035
:1033300025FF0BC040E050E066E070E00E94B11B4A
:103340008091E8008E778093E8000895CF93DF9313
:1033500021E02093E9002FEF3091E800215035FD66
:1033600006C035ED3A95F1F700002111F5CF209117
:10337000E80025FF14C0EC0140E050E068E070E098
:103380000E94B11B8091E8008E778093E80088E06E
:10339000FE01A3E6B2E001900D928A95E1F7DF917C
:1033A000CF910895809360027093620260936102EE
:1033B00080918B02843001F582E08093E9008FEFE9
:1033C0009091E800815095FD06C095ED9A95F1F732
:1033D00000008111F5CF8091E80085FF0DC040E02D
:1033E00050E063E070E080E692E00E94B11B8091C3
:1033F000E8008E778093E8000895BC0184E00C9487
:10340000D219BC0183E00C94D21980918A028111F7
:1034100009C00E94421D0E949F1D8091E2008460AD
:103420008093E200089510928A0208950C948E18F9
:103430006091870281E0611101C080E00C947918ED
:1034400090918B0281E0943009F080E060918702D6
:103450000C947E1842E061EC81E00E94BB1C42E2C9
:1034600061EC82E00E94BB1C90918B0281E0943061
:1034700009F080E0609187020C94871880918D029A
:10348000833009F461C030F4813071F0823009F486
:103490009AC008958A3009F486C08B3009F46CC054
:1034A000893009F0A8C020C080918C02813A09F0CF
:1034B000A2C08091E800877F8093E800809190020D
:1034C00090919102892B21F468E083E692E003C099
:1034D00060E080E090E070E00E94FC1B8091E800DA
:1034E0008B778093E800089580918C02813209F0F7
:1034F00082C08091900290919102029708F07BC067
:103500008091E800877F8093E8008091E80082FD49
:1035100005C080918B028111F8CF6DC02091F3001E
:103520008091F20090E0922B029731F48091F100AB
:10353000813011F0863021F48091F10080936B028C
:103540008091E8008B7753C080918C02813A09F01A
:1035500052C08091900290919102892B09F04BC04A
:103560008091E800877F8093E8008091E80080FFE9
:10357000FCCF8091180136C080918C028132D9F540
:103580008091900290919102892BA9F58091E80099
:10359000877F8093E8000E94F01C80918E028093C8
:1035A00018010C94090780918C02813221F58091D9
:1035B000E800877F8093E8000E94F01C80918F02D2
:1035C00080936C02089580918C02813AA1F48091DD
:1035D000E800877F8093E8008091E80080FFFCCFBF
:1035E00080916C028093F1008091E8008E77809347
:1035F000E8000C94F01C089584B7877F84BF0FB651
:10360000F894A89580916000886180936000109282
:1036100060000FBE90E080E80FB6F89480936100E0
:10362000909361000FBE0C9489180E94421D0E9465
:103630009F1DE2EEF0E080818460808378940C949A
:1036400034208CE091E00C94D31780918B0285306C
:10365000A9F480918B02853079F40E94DA18809168
:1036600089028823B1F30E949B18882391F30E945A
:103670009B1B0E940907EDCF0C940519089508952E
:103680000C94421B292F332723303105C9F060F4F5
:103690002130310581F02230310509F044C08BE33F
:1036A00090E026E532E043C021323105E1F02232DC
:1036B000310549F138C082E190E021E932E037C0BC
:1036C00099278130910549F028F0029761F5E4E0EF
:1036D000F2E005C0E2E5F2E002C0EEE3F2E0849140
:1036E00090E09F0124C06115710541F061307105C2
:1036F000D1F489E090E021E832E019C089E090E05F
:1037000028E632E014C06115710541F061307105A1
:1037100051F48BE790E023EA32E009C080E490E0C6
:103720002EE133E004C080E090E020E030E0FA01D8
:1037300031832083089580E189BD82E189BD09B488
:1037400000FEFDCF8091D8008F7D8093D8008091BE
:10375000E00082608093E0008091E00081FDFCCF7A
:103760000895CF92DF92EF92FF920F931F93CF9322
:10377000DF93EC018B017A010E940F1D811133C090
:10378000E114F10439F0F70180819181081B190BD4
:10379000C80FD91FC12CD12C0115110519F1809129
:1037A000E80085FD16C08091E8008E778093E800E0
:1037B000E114F10449F0F70180819181C80ED91E0E
:1037C000D182C08285E00FC00E940F1D882321F3A3
:1037D0000AC089918093F10001501109FFEFCF1ABF
:1037E000DF0ADACF80E0DF91CF911F910F91FF9038
:1037F000EF90DF90CF900895209192023091930244
:103800002617370748F06115710539F42091E80053
:103810002E772093E80001C0B901FC0120E061157A
:10382000710579F180918B028823F1F18530F1F1F6
:103830008091E80083FD3CC08091E80082FD2EC0AD
:103840008091E80080FFEBCF2091F3008091F2009F
:1038500090E0922B6115710551F08830910538F494
:1038600021912093F100615071090196F3CF21E07D
:10387000089709F020E08091E8008E778093E800B7
:10388000CECF2111CFCF0AC080918B02882361F067
:10389000853061F08091E80083FD0AC08091E800E6
:1038A00082FFF2CF80E0089582E0089583E00895DA
:1038B00081E00895209192023091930226173707F4
:1038C00048F06115710539F42091E8002E772093B6
:1038D000E80001C0B901FC0120E06115710591F11A
:1038E00080918B02882309F440C0853009F43FC0E1
:1038F0008091E80083FD3DC08091E80082FD2FC0EB
:103900008091E80080FFE9CF2091F3008091F200E0
:1039100090E0922B6115710559F08830910540F4C3
:1039200024912093F1003196615071090196F2CFF4
:1039300021E0089709F020E08091E8008E778093DD
:10394000E800CBCF2111CCCF0AC080918B02882315
:1039500061F0853061F08091E80083FD0AC08091BC
:10396000E80082FFF2CF80E0089582E0089583E0CE
:10397000089581E00895982F973068F59093E900B5
:10398000981739F07091EC002091ED005091F00003
:1039900003C0242F762F50E021FD02C09F5FECCFA3
:1039A0003091EB003E7F3093EB003091ED003D7F96
:1039B0003093ED003091EB0031603093EB00709369
:1039C000EC002093ED005093F0002091EE0027FDD5
:1039D000E5CF80E008958F708093E90081E008953D
:1039E00080918C0287FF11C08091E80082FD05C0A4
:1039F00080918B028111F8CF11C08091E8008B7704
:103A00000BC080918B02882349F08091E80080FFF1
:103A1000F8CF8091E8008E778093E8000895209198
:103A2000E4003091E50095E64091EC00842F817030
:103A300040FF23C08091E80080FD1DC080918B0273
:103A4000882399F0853099F08091EB0085FD11C0B5
:103A50004091E4005091E5002417350729F3915077
:103A600011F09A01E1CF84E0089582E0089583E0A7
:103A7000089581E0089580E008954091E80042FFB4
:103A8000DDCF08950E94B01D0E94B81DE0EEF0E069
:103A9000808181608083E8EDF0E080818F77808392
:103AA00019BCA7EDB0E08C918E7F8C9380818F7EC6
:103AB000808310928A0208950F931F93CF93DF9310
:103AC0000E94B01D0E94B81DC8EDD0E088818F779C
:103AD000888388818068888388818F7D888319BCEA
:103AE00010928B0210928702109289021092880223
:103AF00000EE10E0F80180818B7F808388818160F7
:103B0000888342E060E080E00E94BB1CE1EEF0E0D0
:103B100080818E7F8083E2EEF0E08081816080830F
:103B2000808188608083F80180818E7F8083888196
:103B300080618883DF91CF911F910F910895E8ED07
:103B4000F0E080818F7E8083E7EDF0E0808181600E
:103B5000808384E082BF81E080938A020C945C1DA4
:103B6000E8EDF0E080818E7F80831092E20008957E
:103B70001092DA001092E10008951F920F920FB692
:103B80000F9211242F933F934F935F936F937F93E3
:103B90008F939F93AF93BF93EF93FF938091E10037
:103BA00082FF0BC08091E20082FF07C08091E1009C
:103BB0008B7F8093E1000E9433208091DA0080FFA8
:103BC0001FC08091D80080FF1BC08091DA008E7FDB
:103BD0008093DA008091D90080FF0DC080E189BD1B
:103BE00082E189BD09B400FEFDCF81E080938B02A4
:103BF0000E94051A05C019BC10928B020E94131A6C
:103C00008091E10080FF19C08091E20080FF15C023
:103C10008091E2008E7F8093E2008091E2008061DB
:103C20008093E2008091D80080628093D80019BC14
:103C300085E080938B020E94181A8091E10084FF36
:103C400030C08091E20084FF2CC080E189BD82E118
:103C500089BD09B400FEFDCF8091D8008F7D80938F
:103C6000D8008091E1008F7E8093E1008091E20096
:103C70008F7E8093E2008091E20081608093E20079
:103C800080918702882311F084E007C08091E300CF
:103C900087FD02C081E001C083E080938B020E9417
:103CA000201A8091E10083FF29C08091E20083FF08
:103CB00025C08091E100877F8093E10082E08093BE
:103CC0008B02109287028091E1008E7F8093E10049
:103CD0008091E2008E7F8093E2008091E20080611B
:103CE0008093E20042E060E080E00E94BB1C809193
:103CF000F00088608093F0000E94161AFF91EF9107
:103D0000BF91AF919F918F917F916F915F914F91F3
:103D10003F912F910F900FBE0F901F9018951F92FB
:103D20000F920FB60F9211242F933F934F935F93EF
:103D30006F937F938F939F93AF93BF93CF93DF93B3
:103D4000EF93FF93C091E900CF708091EC00D82FE2
:103D5000D17080FDD0E81092E9008091F000877F5B
:103D60008093F00078940E94D31E1092E900809115
:103D7000F00088608093F000CD2BCF70C093E900F5
:103D8000FF91EF91DF91CF91BF91AF919F918F9173
:103D90007F916F915F914F913F912F910F900FBE47
:103DA0000F901F9018951F93CF93DF93CDB7DEB779
:103DB000AA970FB6F894DEBF0FBECDBFECE8F2E0D5
:103DC0008091F100819322E0E439F207C9F70E9463
:103DD0003E1A8091E80083FF2EC180918C02909161
:103DE0008D02492F50E04A30510508F024C1FA01F4
:103DF000EE59FF4F0C946320803821F0823809F08F
:103E00001AC108C08091880290918902992389F093
:103E100082600FC0809190028F70873008F00BC1D4
:103E20008093E9008091EB0085FB882780F9109250
:103E3000E9009091E800977F9093E8008093F1006B
:103E40001092F100D1C0282F2D7F09F0F4C08823F3
:103E500019F0823061F0EFC080918E02813009F05C
:103E6000EAC0933009F080E0809389022EC08091EF
:103E70008E0281112AC0809190028F702FEF280F3F
:103E8000263008F0D8C08093E9002091EB0020FF95
:103E90001CC0933021F48091EB00806214C090919B
:103EA000EB0090619093EB0021E030E0A90102C0AB
:103EB000440F551F8A95E2F74093EA001092EA00FA
:103EC0008091EB0088608093EB001092E900809174
:103ED000E800877F8093E8000E94F01CACC081114D
:103EE000AAC010918E021F778091E3008078812B09
:103EF0008093E3008091E800877F8093E8000E9430
:103F0000F01C8091E80080FFFCCF8091E300806886
:103F10008093E300111102C082E001C083E080932E
:103F20008B0289C08058823008F085C080918E0253
:103F300090918F028C3D53E0950779F583E08A8359
:103F40008AE289834FB7F894DE01139620E03EE0C1
:103F500051E2E32FF0E050935700E49120FF03C0BB
:103F6000E295EF703F5FEF708E2F90E0EA3010F037
:103F7000C79601C0C0968D939D932F5F243149F75A
:103F80004FBF8091E800877F8093E8006AE270E08D
:103F9000CE0101960E94FC1B16C0609190027091A8
:103FA0009102AE014F5F5F4F0E94401BBC01892B05
:103FB00009F441C09091E800977F9093E8008981CF
:103FC0009A810E945A1C8091E8008B778093E800C8
:103FD00032C0803881F58091E800877F8093E800C7
:103FE000809187028093F1008091E8008E7772CFF4
:103FF000811121C080918E0290918F0299270297A2
:10400000D4F48091E800877F8093E80080918E024D
:10401000809387020E94F01C80918702811106C064
:104020008091E30087FD02C081E001C084E08093BD
:104030008B020E942A1A8091E80083FF0AC08091B7
:10404000E800877F8093E8008091EB008062809396
:10405000EB00AA960FB6F894DEBF0FBECDBFDF917E
:10406000CF911F9108950895CF9380918B0288235B
:10407000A1F0C091E900CF709091EC00892F817080
:1040800090FD80E8C82B1092E9008091E80083FD44
:104090000E94D31ECF70C093E900CF91089597FB83
:1040A000072E16F4009407D077FD09D00E946920EE
:1040B00007FC05D03EF4909581959F4F089570952B
:1040C00061957F4F0895EE0FFF1F0590F491E02D4D
:1040D0000994AA1BBB1B51E107C0AA1FBB1FA6174F
:1040E000B70710F0A61BB70B881F991F5A95A9F7A1
:1040F00080959095BC01CD010895FB01DC0104C0C1
:104100008D910190801921F441505040C8F7881BCF
:10411000990B0895F999FECF92BD81BDF89A992720
:1041200080B50895A8E1B0E042E050E00C94BE20D4
:10413000262FF999FECF92BD81BDF89A019700B460
:10414000021639F01FBA20BD0FB6F894FA9AF99A00
:104150000FBE08950396272F0E9499200E94982051
:10416000252F0E949920242F0C9499200196272F07
:104170000E9499200C949820DC01CB01FC01F99954
:10418000FECF06C0F2BDE1BDF89A319600B40D92A3
:0C41900041505040B8F70895F894FFCF5C
:10419C00C8002002280850011E0A14018319A61910
:1041AC008719011AFD19861901E200E900EA00B528
:1041BC0000B600B700CD008301CC008A01920194B7
:1041CC00012102230224022502260227022A02B31D
:1041DC0000B4006F007000818283E200E900EA0005
:1041EC00B500B600B700CD008301CC008A01920166
:1041FC0094012102230224022502260227022A020C
:10420C00B300B4006F007000818283F0F1F4F5F616
:10421C00F76766363534979694C63790919293002B
:10422C00FF0100010000FFFF0000010001FF000082
:00000001FF
